:0200000480007A
:10000000171800001308480097180000938888000C
:100010008320080003510800835128000342F8FFA1
:100020008342080003431800834328000344380038
:1000300023A0180023A2280023A4380023A64800E8
:1000400023A8580023AA680023AC780023AE8800B8
:1000500017150000130505FC97150000938585FD15
:10006000370610F01306C6F26306B5028326C500F4
:100070002320D600832685002320D6008326450032
:100080002320D600832605002320D6001305050172
:100090006FF09FFD370510F0130505F223200500D2
:0400A000000000005C
:10100000EFCDAB8967452301000000000000000020
:10101000FFFFFFFFFFFFFFFFFFFFFFFFFFFFFFFFE0
:10102000FFFFFFFFFFFFFFFFFFFFFFFFFFFFFFFFD0
:040000058000000077
:00000001FF
